:020000040000FA
:0600000091EF31F0120047
:0620000091EF31F0120027
:0620080051EF30F0120060
:06201800AEEF30F01200F3
:02202A000000B4
:04202C008150020BD2
:1020300005E100016151040B01E061818150040B55
:1020400005E100016151080B01E06183120075C0D8
:102050009AF000019A5102E177C09AF076519A27DE
:10206000020E9A5D02E2020E9A6F9A51630802E232
:10207000630E9A6F69819AC074F09A51F66EF76A8E
:10208000D890F636F736C30EF6265E0EF722090014
:10209000F5CF7AF00A00F5CF7BF07B510001E40325
:1020A000F3CF7CF0F4CF7DF000017A510001E4031E
:1020B000F3CF9BF0F45000017C27FF0E0001E403F6
:1020C000F3CF9DF000017B519D03F3CF7EF0F4CF61
:1020D0007FF07A519D03F3CF9CF0F4507E277DAFC3
:1020E0000DD07C697D697A517A257E6F7B517B2189
:1020F0007F6F7C517E5F7D517F5B37D07FAF0DD08E
:102100007E697F697A517A257C6F7B517B217D6F57
:102110007E517C5F7F517D5B12D07C517C277D514D
:102120007D239BAF03D07C2B000E7D237E517E2729
:102130007F517F239CAF03D07E2B000E7F237C6DCD
:102140007D1F000E7D237E6D7F1F7F237A6D7B1F99
:102150007B2380517C5D826F81517D59836F7E51DD
:102160008025846F7F518121856F1200D9CFE6FFD2
:10217000E1CFD9FFFE0EDBCF75F069DFE552E7CF87
:10218000D9FF1200D9CFE6FFE1CFD9FFFE0EDB5019
:102190000001775D09E06A81FE0EDBCF77F073A75F
:1021A00003D0DBCF75F053DFE552E7CFD9FF120044
:1021B000D9CFE6FFE1CFD9FF020EE1260001896BFE
:1021C0008A6B8B6B8C6B050ED56EF294F28A766BF4
:1021D0008D6B8E6B8F6B906B916B926B626B636B85
:1021E000646B656B666B676B686B996B696B6B6B2C
:1021F000736B7387936B6C6B6E6B6D6B876BE7C0E8
:1022000094F0E8C095F0E9C097F0EAC098F00001BA
:10221000A151EA6A940FE96E000EEA22EFCF98F01E
:1022200098C080F00001816B80BF81695E0E8103E0
:10223000F3CF81F08003F3CF80F0F45081278051F9
:102240007C5D826F81517D59836F7E518025846FC3
:102250007F518121856F0001A151F76A8B0FF66EC6
:102260005F0EF7220800F5CF6FF0A151F76A8F0FCC
:10227000F66E5F0EF7220800F5CF70F0A151F76AF5
:10228000930FF66E5F0EF7220800F5CF71F0A151A3
:10229000F76A970FF66E5F0EF7220800F5CF72F01F
:1022A000F090F092F19AF198F086F0880001606B5E
:1022B000616B6C6B020EE15C02E2E16AE552E16E79
:1022C000E552E7CFD9FF12000001E351070B0408E4
:1022D00003E1F090F09279D1F0A003D00001608387
:1022E00002D000016093766B8D6B8E6B8F6B906B61
:1022F000AEDE00016C5166E10001E55123E0F0A083
:1023000005D000016087616B618704D00001609790
:10231000616B61850001E3AF05D00001715180124E
:10232000725181120001450E786F796979C0D7FF2B
:1023300078C0D6FFD58E010E6C6FE5C086F0020E18
:102340006E6F3CD00001E3AF05D0000171518012E7
:1023500072518112F0A00FD00001616B6187608122
:102360000001E3A704D00001050E866F03D0000131
:10237000010E866F0ED00001616B618560910001D6
:10238000E3A704D00001010E866F03D00001050E03
:10239000866F020E6C6F010E6D6F82C078F083C085
:1023A00079F079C0D7FF78C0D6FFD58E6F518012F3
:1023B000705181127CC078F07DC079F06781F09017
:1023C000F09203D1030E6C5D41E1EB0E80166F0EAF
:1023D0008116D59EF294896B8A6B8B6B8C6B606BCC
:1023E000F0A00ED0616B618760810001E3A704D08B
:1023F0000001050E866F03D00001010E866F0DD01F
:10240000616B618560910001E3A704D00001010EBA
:10241000866F03D00001050E866F020E6C6F010EF1
:102420006D6F82C078F083C079F079C0D7FF78C033
:10243000D6FFD58E6F518012705181127CC078F01A
:102440007DC079F06781F090F092BFD0040E6C5D92
:1024500036E1F0A00ED0616B618760810001E3A7D7
:1024600004D00001050E866F03D00001010E866FB7
:102470000DD0616B618560910001E3A704D000017C
:10248000010E866F03D00001050E866F020E6C6F81
:10249000010E6D6F82C078F083C079F079C0D7FFEC
:1024A00078C0D6FFD58E6F518012705181127CC0DA
:1024B00078F07DC079F06781F090F09286D0050EBB
:1024C0006C5D40E1EB0E80166F0E8116D59EF29486
:1024D00073936B81606BF0A00ED0616B618760813C
:1024E0000001E3A704D00001050E866F03D00001B0
:1024F000010E866F0DD0616B618560910001E3A7CD
:1025000004D00001010E866F03D00001050E866F16
:10251000020E6C6F010E6D6F82C078F083C079F08F
:1025200079C0D7FF78C0D6FFD58E6F518012705119
:1025300081127CC078F07DC079F06B816781F0906A
:10254000F09243D0060E6C5D36E1F0A00ED0616BC8
:10255000618760810001E3A704D00001050E866F4A
:1025600003D00001010E866F0DD0616B6185609113
:102570000001E3A704D00001010E866F03D0000123
:10258000050E866F020E6C6F010E6D6F82C078F0C3
:1025900083C079F079C0D7FF78C0D6FFD58E6F5150
:1025A0008012705181127CC078F07DC079F0678113
:1025B000F090F0920AD0050E6C5D05E1020E6E6F90
:1025C000F090F09202D0F090F092120000018A5147
:1025D00052E08FA103D08DC076F039DD8EC08DF032
:1025E00090C08FF08CC08BF0F00E00018A5D20E36C
:1025F0007AC078F07BC079F079C0D7FF78C0D6FF79
:10260000D58E030E6C6F040E6D6FF00E8A5D0BE1BC
:102610000001E3A904D00001080E866F03D0000179
:10262000060E866F03D00F0E8A15866F64811ED04A
:102630006F5180127051811282C078F083C079F09E
:1026400079C0D7FF78C0D6FFD58E7CC078F07DC02A
:1026500079F0030E6C6F010E6D6F8AA103D0050E29
:10266000866F01D0866F8A417F0B896F8A6B8C6B76
:102670006381010E02D0000E00D01200D59EF294AC
:102680000001860705E079C0D7FF78C0D6FFD58E58
:102690006C51040A01E198D2040A01E195D2060ABC
:1026A00001E184D2030A01E15BD2060A01E1D3D140
:1026B000010A01E18CD0030A23E0060A01E085D279
:1026C00086511EE1D70E8016B70E81166C6B000185
:1026D000E55116E00001E3AF05D000017151801211
:1026E000725181120001450E786F796979C0D7FF68
:1026F00078C0D6FFD58E010E6C6FE5C086F065D22E
:102700000001865163E1020E6E5D33E160A70ED0D9
:10271000616B618760810001E3A704D00001050EB1
:10272000866F03D00001010E866F0DD0616B61854D
:1027300060910001E3A704D00001010E866F03D071
:102740000001050E866F020E6C6F010E6D6F82C068
:1027500078F083C079F079C0D7FF78C0D6FFD58EE6
:102760006F518012705181127CC078F07DC079F079
:102770002CD2030E6E5D0AE129DF000906E1D70EB7
:102780008016B70E811600016C6B1FD2050E6E5DB0
:1027900012E16F51801270518112460E786F240E33
:1027A000796F79C0D7FF78C0D6FFD58E050E6C6FD4
:1027B000640E866F0AD287A103D0040E6C6F05D217
:1027C000D70E8016B70E81166C6BFFD1FED16D054A
:1027D00010E186510DE182C078F083C079F079C0B4
:1027E000D7FF78C0D6FFD58E020E6D6F010E866FB3
:1027F000ECD1020E6D5D28E1EB0E80166F0E811696
:1028000084C078F085C079F079C0D7FF78C0D6FF52
:10281000D58E16EC10F00001030E6D6F020E866F60
:102820007451140806E30001E351400B02E100017A
:10283000618500017451270806E30001E351400B54
:1028400002E100016187C1D1030E6D5D01E003D19A
:10285000865101E0ECD00001E3AB0BD08150020BBC
:1028600008E08150040B05E000016051040B01E019
:10287000616B00016185618716EC10F0000161A1B8
:1028800091D061A36AD060850001E351070B030A70
:1028900054E0010A43E0030A22E0010A01E05CD0AF
:1028A000000160A10ED0616B618560910001E3A71A
:1028B00004D00001010E866F03D00001050E866F63
:1028C0000DD0616B618760810001E3A704D0000136
:1028D000050E866F03D00001010E866F3DD000010A
:1028E00060A30ED0616B618760810001E3A704D013
:1028F0000001050E866F03D00001010E866F0DD01A
:10290000616B618560910001E3A704D00001010EB5
:10291000866F03D00001050E866F1ED00001616B2B
:10292000618760810001E3A704D00001050E866F76
:1029300003D00001010E866F0FD00001616B61852D
:1029400060910001E3A704D00001010E866F03D05F
:102950000001050E866F00D00ED06095616B618717
:1029600060810001E3A704D00001050E866F03D04B
:102970000001010E866F0001020E6C6F010E6D6F7B
:1029800082C078F083C079F079C0D7FF78C0D6FFD5
:10299000D58E6F518012705181127CC078F07DC04D
:1029A00079F044D061A324D06095616B618560911A
:1029B0000001E3A704D00001010E866F03D00001DF
:1029C000050E866F020E6C6F010E6D6F82C078F07F
:1029D00083C079F079C0D7FF78C0D6FFD58E6F510C
:1029E0008012705181127CC078F07DC079F01ED0C9
:1029F00060950001E6510EE00001450E786F79699F
:102A000079C0D7FF78C0D6FFD58E060E6C6FE6C0B2
:102A100086F00CD00001658187A103D0040E6C6F95
:102A200005D0D70E8016B70E81166C6B13D074517B
:102A3000290806E30001E351400B02E10001618532
:102A4000000174512B0806E30001E351400B02E141
:102A500000016187BAD0865101E081D06D050EE199
:102A600082C078F083C079F079C0D7FF78C0D6FFF4
:102A7000D58E020E6D6F010E866FA7D0020E6D5DB2
:102A800012E1EB0E80166F0E811684C078F085C0BF
:102A900079F079C0D7FF78C0D6FFD58E030E6D6F61
:102AA000020E866F92D0030E6D5D2CE189051CE04D
:102AB0006F5180127051811282C078F083C079F01A
:102AC00079C0D7FF78C0D6FFD58E7CC078F07DC0A6
:102AD00079F0010E6D6F89A103D0050E866F01D0CC
:102AE000866F899189430DD07AC078F07BC079F0E8
:102AF00079C0D7FF78C0D6FFD58E040E866F6D6F74
:102B0000648163D0040E6D5D2AE160DD000927E178
:102B10000001766B8D6B8E6B8F6B906B27EC10F0DA
:102B2000000165810001E6510EE00001450E786F5D
:102B3000796979C0D7FF78C0D6FFD58E060E6C6F45
:102B4000E6C086F00CD00001658187A103D0040E99
:102B50006C6F05D0D70E8016B70E81166C6B35D012
:102B6000865123E1EB0E80166F0E811673936B81F5
:102B70000001E6510EE00001450E786F796979C0D9
:102B8000D7FF78C0D6FFD58E060E6C6FE6C086F0F4
:102B90000CD00001658187A103D0040E6C6F05D0B5
:102BA000D70E8016B70E81166C6B0FD086510BE1D5
:102BB000658187A103D0040E6C6F05D0D70E8016F7
:102BC000B70E81166C6B01D000D012000001E351EA
:102BD000070B040803E016EC10F063D0070E0001A9
:102BE0006C5D01E15ED081A225D099B15AD0EB0E87
:102BF00080166F0E81160001E6510EE00001450EB1
:102C0000786F796979C0D7FF78C0D6FFD58E060E68
:102C10006C6FE6C086F00CD00001658187A103D0FF
:102C2000040E6C6F05D0D70E8016B70E81166C6B34
:102C3000998137D099A135D0D59EF294996B766B56
:102C40008D6B8E6B8F6B906B27EC10F0030E000179
:102C50006C5D05E1896B8A6B8B6B8C6B6781050EF4
:102C60006C5D04E1D59EF29473936B816C5106E028
:102C7000040E6C5D03E0060E6C5D01E167810001EE
:102C8000E3AF05D000017151801272518112000131
:102C9000020E6C6F010E6D6F6F51801270518112B8
:102CA00000D01200D9CFE6FFE1CFD9FF200EF36E9E
:102CB000FE0EDBCFF4FFF350F45C01E27DD0FE0E9C
:102CC000DB50600801E278D000018A5103E0020E77
:102CD000916F71D0FE0EDB50E00FF76A820FF66E37
:102CE0005E0EF7220800F5CF8AF08A5103E1010E4B
:102CF000916F61D0F29E020E6C5D0DE000019E515D
:102D0000020B09E100016C0503E0070E6C5D07E1B1
:102D1000020E6E5D04E100018A6B888349D0FE0ECD
:102D2000DBCF8CF06C511BE10001E55118E0000194
:102D3000E3AF05D000017151801272518112000180
:102D4000450E786F796979C0D7FF78C0D6FFD58EE8
:102D5000010E6C6FE5C086F0030E6E6F29D0000186
:102D60006C0503E0070E6C5D07E1050E6E5D01E189
:102D70006B81030E6E6F1CD073A302D073936B81B3
:102D80006C5108E10001E3AF05D0000171518012E0
:102D90007251811200016C5109E0040E6C5D06E075
:102DA000050E6C5D03E0060E6C5D02E1E6EC12F0D0
:102DB000F28E0001916B03D00001010E916FE5527C
:102DC000E7CFD9FF1200D9CFE6FFE1CFD9FFE65216
:102DD000F29E00018A5103E1030E926F2DD0200E66
:102DE000F36EFE0EDBCFF4FFF350F45C1BE3FE0E3C
:102DF000DB50600817E3FE0EDB50E00FF76A820F2E
:102E0000F66E5E0EF7220800F550DF6EDF5003E12C
:102E1000010E926F06D0DFCF8AF0FE0EDBCF8CF072
:102E2000926B0AD0FE0EDB5005E18A6B8C6B926BC5
:102E3000668102D0010E926FF28EE552E552E7CF25
:102E4000D9FF1200D9CFE6FFE1CFD9FFE652FE0E3F
:102E5000DB50DF6EF29ED9CFE9FFDACFEAFFEF5009
:102E6000020B53E000016C51070A49E0030A34E009
:102E7000020A32E0060A01E048D073830001E551FE
:102E800018E00001E3AF05D00001715180127251CA
:102E900081120001450E786F796979C0D7FF78C03B
:102EA000D6FFD58E010E6C6FE5C086F0050E6E6FF5
:102EB00012D000016F51801270518112460E786F4E
:102EC000240E796F79C0D7FF78C0D6FFD58E050E56
:102ED0006C6F640E866F19D073836F5180127051BE
:102EE0008112460E786F240E796F79C0D7FF78C0B3
:102EF000D6FFD58E050E6C6F640E866F06D06E51B0
:102F000003E1050E6E6F738300D0D9CFE9FFDACFEE
:102F1000EAFFEF50010B3CE0050E00016C5D25E17E
:102F2000EB0E80166F0E8116D59EF29473930001FE
:102F3000E6510EE00001450E786F796979C0D7FF40
:102F400078C0D6FFD58E060E6C6FE6C086F00CD02A
:102F50000001658187A103D0040E6C6F05D0D70EE8
:102F60008016B70E81166C6B13D06C0511E1050E3F
:102F70006E5D0EE17393D59EF294658187A103D0B7
:102F8000040E6C6F05D0D70E8016B70E81166C6BD1
:102F9000D9CFE9FFDACFEAFFEF50080B02E00001DA
:102FA0007387D9CFE9FFDACFEAFFEF50040B02E0D5
:102FB00000017397F28EE552E552E7CFD9FF120078
:102FC000D9CFE6FFE1CFD9FFF29E00018A5105E09B
:102FD000FE0EDBCF8EF0908104D0FE0EDBCF8DF0A5
:102FE0008F81F28E00D0E552E7CFD9FF1200F29E1A
:102FF000030E00016C5D03E0050E6C5D2DE1EB0E30
:1030000080166F0E8116D59EF294766B8D6B8E6B4B
:103010008F6B906B27EC10F0000165810001E65189
:103020000EE00001450E786F796979C0D7FF78C04E
:10303000D6FFD58E060E6C6FE6C086F00CD0000170
:10304000658187A103D0040E6C6F05D0D70E801662
:10305000B70E81166C6B13D06C0511E1020E6E5D1C
:103060000EE0D59EF2946581658187A103D0040EA0
:103070006C6F05D0D70E8016B70E81166C6B896BFE
:103080008A6B8B6B8C6B7393F28E120000016C5108
:1030900037E0060E6C5D03E1070E6C6F31D0EB0E6E
:1030A00080166F0E8116D59EF294050E6C5D02E1BE
:1030B00073936B81030E6C5D0FE188856581766B80
:1030C0008D6B8E6B8F6B906B27EC10F00001658120
:1030D000896B8A6B8B6B8C6B450E786F796979C0C5
:1030E000D7FF78C0D6FFD58E070E6C6F6E6B0001D0
:1030F000E65103E0E6C086F003D00001050E866FBE
:103100000001A151F76A8B0FF66E5F0EF7220800DF
:10311000F5CF6FF0A151F76A8F0FF66E5F0EF722B1
:103120000800F5CF70F0A151F76A930FF66E5F0EAD
:10313000F7220800F5CF71F0A151F76A970FF66EEC
:103140005F0EF7220800F5CF72F0A151EA6A940FE2
:10315000E96E000EEA22EFCF98F098C080F00001EF
:10316000816B80BF81695E0E8103F3CF81F08003A4
:10317000F3CF80F0F450812780517C5D826F8151C4
:103180007D59836F7E518025846F7F518121856FAA
:103190001200F29E000171518012725181128781DA
:1031A0006C511EE10001E55118E00001E3AF05D0CC
:1031B000000171518012725181120001450E786F29
:1031C000796979C0D7FF78C0D6FFD58E010E6C6FB4
:1031D000E5C086F0040E6E6F03D00001040E6C6F24
:1031E000F28E1200F29E0001876B040E6C5D05E109
:1031F000D70E8016B70E81166C6BF28E1200D9CFE7
:10320000E6FFE1CFD9FFE652FE0EDB50DF6ED9CFED
:10321000E9FFDACFEAFFEF50070B040804E3DFCF42
:10322000E3F00001DD89E552E552E7CFD9FF120056
:10323000D9CFE6FFE1CFD9FFF29EFE0EDBCFE4F05F
:103240000001DD8B27EC10F0F28EE552E7CFD9FFBD
:103250001200D9CFE6FFE1CFD9FFFE0EDBCFE5F0BC
:103260000001DD8DE552E7CFD9FF1200D9CFE6FF8F
:10327000E1CFD9FFFE0EDBCFE6F00001DD8FE55296
:10328000E7CFD9FF1200D9CFE6FFE1CFD9FF030E78
:10329000E126FE0EDB50026ED9CFE9FFDACFEAFF5E
:1032A00002507F0BF36E800EEF14F310EF6EDF9E73
:1032B000FE0EDB50DF6E0001FA510001FB25FF0F0F
:1032C000E76E010EE7CFDBFFD9CFE9FFDACFEAFFE8
:1032D000EF507F0BE76E020EE7CFDBFFFE0EDB50F9
:1032E00007E1F29EECC0FAF0EDC0FBF0F28E3FD0A9
:1032F000020EF36EDBCFF4FFF350F45C04E2020E37
:10330000F36EF3CFDBFF020EDB50630805E2630EC2
:10331000F36E020EF3CFDBFF020EDB50F36E010EF5
:10332000DBCFF4FFF350F45C06E2020EDB50E76EF5
:10333000010EE7CFDBFFF29E020EDBCFFAF0010EAB
:10334000DBCFE6FF020EDB50E552E75C010FFB6FBF
:10335000F28ED9CFE9FFDACFEAFFEF50800B07E01A
:10336000FAC0ECF00001DE8BFBC0EDF0DE8D030E49
:10337000E15C02E2E16AE552E16EE552E7CFD9FF96
:103380001200D9CFE6FFE1CFD9FF030EE126FE0EF2
:10339000DB50DF6ED9CFE9FFDACFEAFFEF507F0BCA
:1033A000E76E010EE7CFDBFF020EFAC0DBFFF36E24
:1033B000010EDBCFF4FFF350F45C03E2DE52020EA9
:1033C000DD6E010EDB50630803E2DE52630EDD6E3C
:1033D000020EDB50F36E010EDBCFF4FFF350F45C12
:1033E00006E2010EDB50E76E020EE7CFDBFFF29E36
:1033F000020EDB500001FA5D010EDBCFE6FF020E8C
:10340000DB50E552E75C010F0001FB6FF28ED9CF74
:10341000E9FFDACFEAFFEF50800B07E0FAC0ECF0EB
:103420000001DE8BFBC0EDF0DE8D030EE15C02E2FD
:10343000E16AE552E16EE552E7CFD9FF12000001E3
:10344000A151EA6A940FE96E000EEA22EFCF98F0DC
:10345000F29E98C080F00001816B80BF81695E0E92
:103460008103F3CF81F08003F3CF80F0F450812704
:1034700080517C5D826F81517D59836F7E518025A3
:10348000846F7F518121856FF28E1200D9CFE6FFC4
:10349000E1CFD9FFE652FE0EDB50DF6ED9CFE9FF58
:1034A000DACFEAFFEF507F0BE8BC80090001946F90
:1034B000C00E945D02E1E7C094F0D9CFE9FFDACF06
:1034C000EAFFEF50800B04E094C0E7F00001DE81DA
:1034D000B6DFE552E552E7CFD9FF1200D9CFE6FFBC
:1034E000E1CFD9FFE652FE0EDB50DF6ED9CFE9FF08
:1034F000DACFEAFFEF507F0BE8BC80090001956F3F
:10350000C00E955D02E1E8C095F0D9CFE9FFDACFB2
:10351000EAFFEF50800B04E095C0E8F00001DE8385
:103520008EDFE552E552E7CFD9FF1200D9CFE6FF93
:10353000E1CFD9FFE652FE0EDB50DF6ED9CFE9FFB7
:10354000DACFEAFFEF507F0BE8BC80090001966FED
:10355000C00E965D02E1E9C096F0D9CFE9FFDACF5F
:10356000EAFFEF50800B04E096C0E9F00001DE8531
:1035700066DFE552E552E7CFD9FF1200D9CFE6FF6B
:10358000E1CFD9FFE652FE0EDB50DF6ED9CFE9FF67
:10359000DACFEAFFEF507F0BE8BC80090001976F9C
:1035A000C00E975D02E1EAC097F0D9CFE9FFDACF0C
:1035B000EAFFEF50800B04E097C0EAF00001DE87DD
:1035C0003EDFE552E552E7CFD9FF120075C093F018
:1035D0000001935100D012000001E45100D012000C
:1035E0000001775100D01200D9CFE6FFE1CFD9FF1B
:1035F000E652DF6A00016C51010A16E0040A10E08D
:10360000060A0AE0010A04E0DF90DF92DF9424D08A
:10361000DF80DF92DF9420D0DF90DF82DF941CD048
:10362000DF80DF82DF9418D06E51050A10E0060AB1
:103630000AE0010A04E0DF90DF92DF940CD0DF8023
:10364000DF92DF9408D0DF90DF82DF9404D0DF8048
:10365000DF82DF9400D000D08A5101E1DF880001D1
:103660009EB3DF86DF5000D0E552E552E7CFD9FFA9
:1036700012000001915100D012000001925100D0BF
:1036800012000001765100D01200D9CFE6FFE1CF41
:10369000D9FFE65273C0DFFFD9CFE9FFDACFEAFFE7
:1036A000EF50020B01E1DF80D9CFE9FFDACFEAFF6B
:1036B000EF50080B01E1DF84DF5000D0E552E55206
:1036C000E7CFD9FF1200000169A106D0696B7551DF
:1036D000935D02E0010E02D0000E00D01200000146
:1036E0006AA103D06A6B010E02D0000E00D0120056
:1036F00000016BA103D06B6B010E02D0000E00D055
:103700001200000163A103D0636B010E02D0000E12
:1037100000D01200000166A103D0666B010E02D03A
:10372000000E00D01200000164A103D0646B010EF2
:1037300002D0000E00D01200000165A103D0656B1D
:10374000010E02D0000E00D01200000167A103D0CC
:10375000676B010E02D0000E00D01200D9CFE6FF39
:10376000E1CFD9FFE652F29E88C0DFFF0001886BEF
:10377000F28EDF5000D0E552E552E7CFD9FF1200BC
:1037800000018B5100D012000001FA5100D012004C
:103790000001FA510001FB25FF0F00D01200D9CF24
:1037A000E6FFE1CFD9FFE65294C0DFFFDF9EDF5096
:1037B00000D0E552E552E7CFD9FF1200D9CFE6FF9E
:1037C000E1CFD9FFE65295C0DFFFDF9EDF5000D08A
:1037D000E552E552E7CFD9FF1200D9CFE6FFE1CF9E
:1037E000D9FFE65296C0DFFFDF9EDF5000D0E552E2
:1037F000E552E7CFD9FF1200D9CFE6FFE1CFD9FFDD
:10380000E65297C0DFFFDF9EDF5000D0E552E55261
:06381000E7CFD9FF120012
:0A381600806A0E0EC16EC10E926EA4
:10382000816A070E936E826A946A966A846A836AD2
:10383000F00E956E848E8C908C948C928C960001F8
:10384000DA6BDB6B0001DA07000EDB5B0001DA519B
:10385000DB1103E000000000F5D7F4EC25F010ECDC
:1038600024F0CEEC2FF0D8EC10F032EC28F0E6EC9F
:103870002EF0120095EC24F00AEC27F0060E010160
:10388000225D03E36D50020B01E003D022D8A1ECCE
:1038900020F01200D9CFE6FFE1CFD9FF04010CAF31
:1038A00003D0F3EC2DF0FAD7FE0EDBCFCAF0FD0EFD
:1038B000DBCFCBF0020EE66ECA0EE66E000EE66EB1
:1038C0005CEC2DF0E552E552E552E552E7CFD9FF29
:1038D0001200020EE66ED20EE66E000EE66E96EC5A
:1038E0002DF0E552E552E5520001C96F020E0001CC
:1038F000C95D02E0A0EF20F00001D251430A02E1CD
:1039000088EF20F0010A01E1F4D3030A01E1E7D3D3
:10391000010A01E1D5D3750A01E1C3D3010A01E12E
:10392000B1D3070A01E1A0D3010A01E193D3030A4D
:1039300001E182D3010A01E170D3130A01E15ED3F0
:10394000010A01E14DD3030A01E13CD3010A01E17F
:103950002BD3730A01E11AD3010A01E109D3030A47
:1039600001E1F8D2010A01E1E7D24F0A01E1D6D222
:10397000010A01E1C5D2030A01E1B9D2010A01E15C
:10398000ADD2070A01E19CD2010A01E18CD2030AFF
:1039900001E17CD2010A01E16BD20F0A01E161D29F
:1039A000010A01E150D2030A01E143D2010A01E117
:1039B00032D2070A01E121D2010A01E111D2030A40
:1039C00001E1FED1010A01E1F2D1180A01E1D0D1F1
:1039D0000A0A01E1C6D1030A01E1BBD1010A01E0F3
:1039E000A6D30001D351430A01E1A1D1010A01E1AB
:1039F00095D1030A01E189D1010A01E17DD1750A5E
:103A000001E171D1010A01E165D1070A01E15AD151
:103A1000010A01E14ED1030A01E143D1010A01E1AA
:103A200037D1130A01E12BD1010A01E11FD1030AA9
:103A300001E113D1010A01E107D1730A01E1FBD0D1
:103A4000010A01E1EFD0030A01E1E3D0010A01E13B
:103A5000D7D04F0A01E1CBD0010A01E1BFD0030A60
:103A600001E1B3D0010A01E1A7D0070A01E19BD02F
:103A7000010A01E190D0030A01E185D0010A01E1C8
:103A800079D00F0A70E0010A65E0030A5CE0010AE0
:103A900051E0070A46E0010A3CE0030A31E0010A6E
:103AA00026E0180A1DE00A0A14E0030A0AE0010AE7
:103AB00001E046D1120EE66EE66AECDEE552E55212
:103AC00047D1010EE66E010EE66EE4DEE552E552E8
:103AD0003FD1E66A020EE66EDDDEE552E55238D1F0
:103AE000E66A080EE66ED6DEE552E55231D1F4EC18
:103AF0001AF0E66E100EE66ECDDEE552E55228D1E4
:103B0000E6EC1AF0E66E110EE66EC4DEE552E55202
:103B10001FD1E3C0E6FF120EE66EBCDEE552E552B1
:103B200017D139EC1BF0E66E130EE66EB3DEE552EC
:103B3000E5520ED13DEC1BF0E66E140EE66EAADEE9
:103B4000E552E55205D1E66A150EE66EA3DEE552B2
:103B5000E552FED045EC1BF0E66E160EE66E9ADEE0
:103B6000E552E552F5D0E66A170EE66E93DEE552B1
:103B7000E552EED041EC1BF0E66E180EE66E8ADEE2
:103B8000E552E552E5D0E5C0E6FF190EE66E82DEAD
:103B9000E552E552DDD0E6C0E6FF1A0EE66E7ADEAB
:103BA000E552E552D5D0ECEC1AF0E66E1B0EE66E4F
:103BB00071DEE552E552CCD0F0EC1AF0E66E1C0E48
:103BC000E66E68DEE552E552C3D0C0EC1BF0E66E4F
:103BD0001D0EE66E5FDEE552E552BAD0C4EC1BF076
:103BE000E66E1E0EE66E56DEE552E552B1D0C8EC2A
:103BF0001BF0E66E1F0EE66E4DDEE552E552A8D0D4
:103C0000CFEC1BF0E66E500EE66E44DEE552E55258
:103C10009FD0DEEC1BF0E66E510EE66E3BDEE55209
:103C2000E55296D0EDEC1BF0E66E520EE66E32DEFB
:103C3000E552E5528DD0FCEC1BF0E66E530EE66EBD
:103C400029DEE552E55284D031EC2FF0E66E200EED
:103C5000E66E20DEE552E5527BD035EC2FF0E66EC5
:103C6000210EE66E17DEE552E55272D039EC2FF0E8
:103C7000E66E220EE66E0EDEE552E55269D03DECB0
:103C80002FF0E66E230EE66E05DEE552E55260D0BB
:103C9000E0EC24F0E66E300EE66EFCDDE552E55217
:103CA00057D0DFC0E6FF310EE66EF4DDE552E55297
:103CB0004FD0E4EC24F0E66E320EE66EEBDDE5521A
:103CC000E55246D0E0C0E6FF330EE66EE3DDE55296
:103CD000E5523ED059EC25F0E66E340EE66EDADDA4
:103CE000E552E55235D085EC25F0E66E350EE66EF0
:103CF000D1DDE552E5522CD04CEC29F0E66E400EB9
:103D0000E66EC8DDE552E55223D050EC29F0E66EB0
:103D1000410EE66EBFDDE552E5521AD082EC29F085
:103D2000E66E420EE66EB6DDE552E55211D0C2EC0B
:103D300029F0E66E430EE66EADDDE552E55208D0A1
:103D4000D3C0E6FF7F0EE66EA5DDE552E55200D05A
:103D5000F7D1010EE66E010EE66E9CDDE552E552EE
:103D6000EFD1E66A020EE66E95DDE552E552E8D146
:103D7000210E0001D35D13E12BEC28F0F1EC2DF0C6
:103D80000001DA6BDB6B0001DA07000EDB5B000180
:103D9000DA51DB1103E000000000F5D7FF00010E4F
:103DA000E66E080EE66E76DDE552E552C9D1F4EC1A
:103DB0001AF0E66E100EE66E6DDDE552E552C0D1EA
:103DC000F29ED3C0E6FFB6EC10F0E552F28EE6ECC0
:103DD0001AF0E66E110EE66E5DDDE552E552B0D1E9
:103DE000D3C0E6FFFFEC18F0E552E3C0E6FF120E89
:103DF000E66E50DDE552E552A3D1D3C0E6FF52ECAA
:103E000016F0E55239EC1BF0E66E130EE66E42DD5D
:103E1000E552E55295D1D3C0E6FFE3EC16F0E5524A
:103E20003DEC1BF0E66E140EE66E34DDE552E55215
:103E300087D1F7EC17F0010EE66E150EE66E2ADD5F
:103E4000E552E5527DD1D3C0E6FF22EC17F0E552F2
:103E500045EC1BF0E66E160EE66E1CDDE552E552F3
:103E60006FD1E66A170EE66E15DDE552E55268D1B0
:103E7000D3C0E6FFE0EC17F0E55241EC1BF0E66E34
:103E8000180EE66E07DDE552E5525AD1D3C0E6FFC3
:103E900029EC19F0E552E5C0E6FF190EE66EFADCF2
:103EA000E552E5524DD1D3C0E6FF36EC19F0E552AC
:103EB000E6C0E6FF1A0EE66EEDDCE552E55240D1B3
:103EC000D3C0E6FF18EC19F0E552ECEC1AF0E66E00
:103ED0001B0EE66EDFDCE552E55232D1F0EC1AF053
:103EE000E66E1C0EE66ED6DCE552E55229D1C0EC3A
:103EF0001BF0E66E1D0EE66ECDDCE552E55220D1DC
:103F0000D3C0E6FF43EC19F0E552C4EC1BF0E66EBB
:103F10001E0EE66EBFDCE552E55212D1D3C0E6FFBD
:103F2000C1EC19F0E552C8EC1BF0E66E1F0EE66E10
:103F3000B1DCE552E55204D1D3C0E6FF46EC1AF0FD
:103F4000E552CFEC1BF0E66E500EE66EA3DCE552B8
:103F5000E552F6D0D3C0E6FF6EEC1AF0E552DEEC87
:103F60001BF0E66E510EE66E95DCE552E552E8D0A8
:103F7000D3C0E6FF96EC1AF0E552EDEC1BF0E66ECE
:103F8000520EE66E87DCE552E552DAD0D3C0E6FF8A
:103F9000BEEC1AF0E552FCEC1BF0E66E530EE66E3A
:103FA00079DCE552E552CCD0D3C0E6FFF1EC2EF03F
:103FB000E55231EC2FF0E66E200EE66E6BDCE5523A
:103FC000E552BED0D3C0E6FF01EC2FF0E55235EC50
:103FD0002FF0E66E210EE66E5DDCE552E552B0D0C4
:103FE000D3C0E6FF11EC2FF0E55239EC2FF0E66E6E
:103FF000220EE66E4FDCE552E552A2D0D3C0E6FFBA
:1040000021EC2FF0E5523DEC2FF0E66E230EE66E2C
:104010004AEC1CF0E552E55293D0D3C0E6FFD2EC57
:1040200024F0E552E0EC24F0E66E300EE66E4AEC49
:104030001CF0E552E55284D0D3C0E6FFA5EC24F095
:10404000E552DFC0E6FF310EE66E4AEC1CF0E552A9
:10405000E55276D0E4EC24F0E66E320EE66E4AECE1
:104060001CF0E552E5526CD0D3C0E6FFB7EC24F06B
:10407000E552E0C0E6FF330EE66E4AEC1CF0E55276
:10408000E5525ED0D3C0E6FFF3EC24F0E55259ECE4
:1040900025F0E66E340EE66E4AEC1CF0E552E55271
:1040A0004FD0D3C0E6FF26EC25F0E55285EC25F095
:1040B000E66E350EE66E4AEC1CF0E552E55240D055
:1040C000D3C0E6FFD2EC28F0E5524CEC29F0E66EC6
:1040D000400EE66E4AEC1CF0E552E55231D050EC51
:1040E00029F0E66E410EE66E4AEC1CF0E552E55210
:1040F00027D0D3C0E6FFEDEC28F0E55282EC29F0A2
:10410000E66E420EE66E4AEC1CF0E552E55218D01F
:10411000D3C0E6FFA3EC28F0E552C2EC29F0E66E2E
:10412000430EE66E4AEC1CF0E552E55209D0D2C0CF
:10413000E6FF7F0EE66E4AEC1CF0E552E55200D039
:10414000120004010CBFCCD078EC1BF000090AE08F
:1041500045EC1BF0E66E160EE66E4AEC1CF0E552DE
:10416000E552BED0AEEC1BF00001DC6FDC5109E083
:10417000DCC0E6FF150EE66E4AEC1CF0E552E55297
:10418000AFD08AEC1BF0000909E0030EE66E170EB3
:10419000E66E4AEC1CF0E552E552A2D081EC1BF031
:1041A00000090AE0C0EC1BF0E66E1D0EE66E4AEC5C
:1041B0001CF0E552E55294D093EC1BF0000909E0A5
:1041C000010EE66E170EE66E4AEC1CF0E552E55263
:1041D00087D09CEC1BF0000909E0020EE66E170E7A
:1041E000E66E4AEC1CF0E552E5527AD0A5EC1BF0E5
:1041F000000909E0040EE66E170EE66E4AEC1CF0AC
:10420000E552E5526DD063EC1BF000090AE0E6ECE4
:104210001AF0E66E110EE66E4AEC1CF0E552E5521D
:104220005FD06FEC1BF000090AE0F0EC1AF0E66ECC
:104230001C0EE66E4AEC1CF0E552E55251D0C6EC7D
:1042400029F000090AE050EC29F0E66E410EE66E16
:104250004AEC1CF0E552E55243D0EAEC24F00009A8
:104260000AE0E4EC24F0E66E320EE66E4AEC1CF056
:10427000E552E55235D00001C5510BE0C5C0E6FF5F
:104280000A0EE66E4AEC1CF0E552E5520001C56BE1
:1042900027D0C6510BE0C6C0E6FF0B0EE66E4AEC17
:1042A0001CF0E552E5520001C66B1AD0C7510BE075
:1042B000C7C0E6FF0C0EE66E4AEC1CF0E552E55274
:1042C0000001C76B0DD0C8510BE0C8C0E6FF0D0E52
:1042D000E66E4AEC1CF0E552E5520001C86B00D0D6
:0242E0001200CA
:0E42E200D9CFE6FFE1CFD9FF0001080EC46F6F
:1042F000FE0EDBAE02D08D8201D08D920000000058
:104300000001C4078D80FE0EDBCFE7FFE79EE74686
:10431000FE0EE7CFDBFF000000008D900001C451CE
:10432000E7E1E552E7CFD9FF12000001B9A507D0B8
:10433000A2C0A6F0A8C0B4F0A9C0B5F03CD0B9A7FF
:1043400007D0A3C0A6F0AAC0B4F0ABC0B5F033D07C
:10435000B8A319D0B8A907D0A5C0A6F0B2C0B4F0D0
:10436000B3C0B5F00FD0B8A507D0A5C0A6F0AEC0B9
:10437000B4F0AFC0B5F006D0A3C0A6F0AAC0B4F0A8
:10438000ABC0B5F018D0B8A907D0A4C0A6F0B0C093
:10439000B4F0B1C0B5F00FD0B8A507D0A4C0A6F056
:1043A000ACC0B4F0ADC0B5F006D0A2C0A6F0A8C0B5
:1043B000B4F0A9C0B5F0C00EB513A651040B06E0C9
:1043C0000001DF51080B02E00001B5890001B65180
:1043D000B41902E1B751B5190AE08992B5C0E6FFF8
:1043E00080DFE552B4C0E6FF7CDFE5528982000140
:1043F000A6A102D08C8001D08C90A6A302D08C8282
:1044000001D08C92A6C0A7F0B4C0B6F0B5C0B7F08A
:104410001200D9CFE6FFE1CFD9FFE6529FC0DFFF00
:10442000F29E00019E6BB9A104D09E91B8B19E830B
:104430000DD0B9A306D09E81A0C0DFFFB8A19E8396
:1044400005D0B8A103D09E81A0C0DFFFA151DF5CE1
:1044500006E0DFCFA1F046EC18F02CEC29F0F28E4C
:104460000001DFA90CD0FC0E82160001A151F76AF1
:104470001A0FF66E630EF7220800F5508212000143
:10448000DFAB0ED00001A151F76A1E0FF66E630E6E
:10449000F7220800F5CFBAF0F29EB4EC2EF0F28EBF
:1044A00000019EA103D08C868C9402D08C848C96C3
:1044B000E552E552E7CFD9FF1200D9CFE6FFE1CFB1
:1044C000D9FFE652DF6A0001B951100B06E1B8517D
:1044D000080B06E09E51020B03E1C9EC18F002D074
:1044E000F2EC18F0E552E552E7CFD9FF12000001D7
:1044F000DF51070B010A01E12ED1030A01E1ADD022
:10450000020A01E08CD10001010EA26F070EA46F18
:10451000020EA36F070EA56F9F51F66EF76AD89033
:10452000F636F736120EF626630EF7220900F5CF9F
:1045300002F00800F5CF03F09F51F66EF76AD890AD
:10454000F636F736020EF626630EF7220900F5500E
:10455000000102100001A86F0900F55000010310CE
:104560000001A96FA051F66EF76AD890F636F736BB
:104570000A0EF626630EF7220900F5CF02F00800B6
:10458000F5CF03F09F51F66EF76AD890F636F736FE
:10459000020EF626630EF7220900F5500001021004
:1045A0000001AC6F0900F550000103100001AD6F70
:1045B000A051F66EF76AD890F636F736020EF62658
:1045C000630EF7220900F5CF02F00800F5CF03F0E3
:1045D0009F51F66EF76AD890F636F7360A0EF62631
:1045E000630EF7220900F550000102100001B06FC0
:1045F0000900F550000103100001B16FA051F66EE3
:10460000F76AD890F636F736120EF626630EF722C2
:104610000900F5CF02F00800F5CF03F0A051F66EC7
:10462000F76AD890F636F736020EF626630EF722B2
:104630000900F550000102100001AA6F0900F550B1
:10464000000103100001AB6FACC0AEF0ADC0AFF025
:10465000B0C0B2F0B1C0B3F0E2D00001050EA26F5D
:10466000070EA46F060EA36F070EA56F9F51F66E7F
:10467000F76AD890F636F736020EF626630EF72262
:104680000900F5CFA8F00A00F5CFA9F0A051F66E09
:10469000F76AD890F636F7360A0EF626630EF7223A
:1046A0000900F5CF02F00800F5CF03F09F51F66E38
:1046B000F76AD890F636F736020EF626630EF72222
:1046C0000900F550000102100001AC6F0900F5501F
:1046D000000103100001AD6FA051F66EF76AD8908B
:1046E000F636F736020EF626630EF7220900F5CFEE
:1046F00002F00800F5CF03F09F51F66EF76AD890EC
:10470000F636F7360A0EF626630EF7220900F55044
:10471000000102100001B06F0900F5500001031004
:104720000001B16FA051F66EF76AD890F636F736F1
:104730000A0EF626630EF7220900F5CFAAF00A004A
:10474000F5CFABF0ACC0AEF0ADC0AFF0B0C0B2F0E2
:10475000B1C0B3F064D00001010EA26FA46F020ECD
:10476000A36FA56F9F51F66EF76AD890F636F736AD
:104770000A0EF626630EF7220900F5CF02F00800B4
:10478000F5CF03F09F51F66EF76AD890F636F736FC
:10479000020EF626630EF7220900F5500001021002
:1047A0000001A86F0900F550000103100001A96F76
:1047B000A8C0ACF0A9C0ADF0A8C0B0F0A9C0B1F0DD
:1047C000A051F66EF76AD890F636F7360A0EF6263E
:1047D000630EF7220900F5CF02F00800F5CF03F0D1
:1047E000A051F66EF76AD890F636F736020EF62626
:1047F000630EF7220900F550000102100001AA6FB4
:104800000900F550000103100001AB6FAAC0AEF023
:10481000ABC0AFF0AAC0B2F0ABC0B3F000D0120092
:10482000E66A5FDDE552E66A5CDDE5528A8A8982E6
:10483000E1C09FF0E2C0A0F09FC0A1F00001B86B02
:10484000BC6BBD6BBE6BB96BBB6BBF6BC06BC16B25
:10485000C26BC36B09D8E0C0E6FF89D8E55247DEDA
:1048600064DDD7DD5DEF22F00001BF5102E0BF073C
:104870000FD083A807D0B9A504D0B995BC810A0E82
:10488000BF6F06D0B9B504D0B985BC810A0EBF6F21
:10489000C05102E0C0070FD083AA07D0B9A704D047
:1048A000B997BC810A0EC06F06D0B9B704D0B987DA
:1048B000BC810A0EC06FC15102E0C1070FD083ACAA
:1048C00007D0B9A104D0B991BD810A0EC16F06D03D
:1048D000B9B104D0B981BD810A0EC16FC25102E0E5
:1048E000C2070FD083AE07D0B9A304D0B993BD815E
:1048F0000A0EC26F06D0B9B304D0B983BD810A0EC7
:10490000C26FC35102E0C3070FD081A007D0B9A97D
:1049100004D0B999BE810A0EC36F06D0B9B904D0CC
:10492000B989BE810A0EC36F12000001BCA102D07A
:10493000BC6BFBDC0001BDA102D0BD6B6ADD0001D8
:10494000BEA102D0BE6BB9DD1200D9CFE6FFE1CF28
:10495000D9FFFE0EDB503F0B0001DF6F0001DD8150
:10496000C6DDE3DC56DDE552E7CFD9FF1200D9CF33
:10497000E6FFE1CFD9FFFE0EDBCFE0F00001DD87DF
:104980008D8000008A9A00008D90110EE66EA9DCE1
:10499000E552E0C0E6FFA5DCE5528A8AE552E7CFA2
:1049A000D9FF1200D9CFE6FFE1CFD9FFFE0EDBCF52
:1049B000B8F0BBDC2EDD81DDE552E7CFD9FF120078
:1049C0000001B85100D01200B9C0BBF00001BB51CA
:1049D00000D012000001BB51B95D02E0010E02D00F
:1049E000000E00D01200D9CFE6FFE1CFD9FFE6528A
:1049F000FE0EDB50DF6ED9CFE9FFDACFEAFFEF50D2
:104A0000100B0BE0D9CFE9FFDACFEAFFEF500F0B25
:104A1000030B0001E16F0001DD83D9CFE9FFDACF9D
:104A2000EAFFEF50200B0DE0F29ED9CFE9FFDACF7D
:104A3000EAFFEF500F0B00019F6FEBDCF28E57DDAA
:104A400074DCE552E552E7CFD9FF1200D9CFE6FF7B
:104A5000E1CFD9FFE652FE0EDB50DF6ED9CFE9FF82
:104A6000DACFEAFFEF50100B0BE0D9CFE9FFDACF36
:104A7000EAFFEF500F0B030B0001E26F0001DD8531
:104A8000D9CFE9FFDACFEAFFEF50200B0DE0F29E1D
:104A9000D9CFE9FFDACFEAFFEF500F0B0001A06F8B
:104AA000B8DCF28E24DD41DCE552E552E7CFD9FFD8
:104AB0001200D9CFE6FFE1CFD9FFE65200019F51A6
:104AC000026ED9CFE9FFDACFEAFF02500F0BF36E87
:104AD000F00EEF14F310EF6E0001E151026ED9CF2A
:104AE000E9FFDACFEAFF02500F0BF36EF346F3460D
:104AF000F346F3460F0EEF14F310EF6EDF5000D0C5
:104B0000E552E552E7CFD9FF1200D9CFE6FFE1CF5A
:104B1000D9FFE6520001A051026ED9CFE9FFDACFEA
:104B2000EAFF02500F0BF36EF00EEF14F310EF6E6E
:104B30000001E251026ED9CFE9FFDACFEAFF02505D
:104B40000F0BF36EF346F346F346F3460F0EEF14E6
:104B5000F310EF6EDF5000D0E552E552E7CFD9FFFA
:024B6000120041
:0E4B6200D9CFE6FFE1CFD9FFFE0EDB50A96EE2
:104B7000A69EA69CA680A85000D0E552E7CFD9FFFC
:104B80001200D9CFE6FFE1CFD9FFFE0EDB50A96EB0
:104B9000FD0EDB50A86EA69EA69CA684550EA76EA1
:104BA000AA0EA76EA682A6B2FED7A69400D0E552A2
:104BB000E7CFD9FF1200D9CFE6FFE1CFD9FFF29EB0
:104BC000FE0EDB50A96EFD0EDB50A86EA69EA69CC5
:104BD000A684550EA76EAA0EA76EA682F28E00D0EE
:104BE000E552E7CFD9FF1200D9CFE6FFE1CFD9FFD9
:104BF000E6520001DD6BDE6BE66AB3DFE5520108C9
:104C000013E1010EE66EADDFE55232080DE1020E52
:104C1000E66EA7DFE552450807E1030EE66EA1DF69
:104C2000E552670801E18BD0010EE66EE66AA9DF66
:104C3000E552E552320EE66E010EE66EA2DFE55257
:104C4000E552450EE66E020EE66E9BDFE552E5523A
:104C5000670EE66E030EE66E94DFE552E552100E27
:104C6000E66E040EE66E8DDFE552E552E66A050E4D
:104C7000E66E87DFE552E552E66AE66882DFE552D6
:104C8000E552E66A060EE66E7CDFE552E552800EDE
:104C9000E66E070EE66E75DFE552E552E66A080E2F
:104CA000E66E6FDFE552E552E66A090EE66E69DFF1
:104CB000E552E552E66A0A0EE66E63DFE552E5521A
:104CC000E66A0B0EE66E5DDFE552E552E66A0C0E13
:104CD000E66E57DFE552E552E66A0D0EE66E51DFED
:104CE000E552E552E66A0E0EE66E4BDFE552E552FE
:104CF000010EE66E0F0EE66E44DFE552E552E66AFF
:104D0000100EE66E3EDFE552E552050EE66E110E20
:104D1000E66E37DFE552E5522D0EE66E120EE66EB8
:104D200030DFE552E552E66A130EE66E2ADFE55201
:104D3000E552E66A140EE66E24DFE552E552040EF3
:104D4000E66E0FDFE5520001DF6F050EE66E09DF4C
:104D5000E5520001E36F060EE66E03DFE552000147
:104D6000E06F070EE66EFDDEE5520001E46F080E0F
:104D7000E66EF7DEE5520001E56F090EE66EF1DE44
:104D8000E5520001E66F0A0EE66EEBDEE552000129
:104D9000E76F0B0EE66EE5DEE5520001E86F0C0EE4
:104DA000E66EDFDEE5520001E96F0D0EE66ED9DE3C
:104DB000E5520001EA6F0E0EE66ED3DEE552000109
:104DC000E16F0F0EE66ECDDEE5520001E26F100ED0
:104DD000E66EC7DEE5520001EB6F110EE66EC1DE36
:104DE000E5520001EC6F120EE66EBBDEE5520001EB
:104DF000ED6F130EE66EB5DEE5520001EE6F140E98
:104E0000E66EAFDEE5520001EF6FE552E552E7CF07
:104E1000D9FF1200A6B21ED10001DDA111D0040EEF
:104E2000E66E9FDEE5520001DF5D07E0DFC0E6FFD2
:104E3000040EE66EC0DEE552E5520001DD910AD1B6
:104E4000DDA911D0050EE66E8CDEE5520001E35DB2
:104E500007E0E3C0E6FF050EE66EADDEE552E55283
:104E60000001DD99F7D0DDA311D00E0EE66E79DEDC
:104E7000E5520001E15D07E0E1C0E6FF0E0EE66EDF
:104E80009ADEE552E5520001DD93E4D0DDA511D0B4
:104E90000F0EE66E66DEE5520001E25D07E0E2C05D
:104EA000E6FF0F0EE66E87DEE552E5520001DD9566
:104EB000D1D0DDA711D0060EE66E53DEE55200011B
:104EC000E05D07E0E0C0E6FF060EE66E74DEE55248
:104ED000E5520001DD97BED0DDAB11D0070EE66EC6
:104EE00040DEE5520001E45D07E0E4C0E6FF070EA6
:104EF000E66E61DEE552E5520001DD9BABD0DDAD33
:104F000011D0080EE66E2DDEE5520001E55D07E0EA
:104F1000E5C0E6FF080EE66E4EDEE552E552000102
:104F2000DD9D98D0DDAF11D0090EE66E1ADEE55298
:104F30000001E65D07E0E6C0E6FF090EE66E3BDE37
:104F4000E552E5520001DD9F85D0DEA911D0100E9B
:104F5000E66E07DEE5520001EB5D07E0EBC0E6FF21
:104F6000100EE66E28DEE552E5520001DE9972D0A1
:104F7000DEAB11D0110EE66EF4DDE5520001EC5D02
:104F800007E0ECC0E6FF110EE66E15DEE552E552D5
:104F90000001DE9B5FD0DEAD11D0120EE66EE1DDCA
:104FA000E5520001ED5D07E0EDC0E6FF120EE66E92
:104FB00002DEE552E5520001DE9D4CD0DEA111D0AB
:104FC0000A0EE66ECEDDE5520001E75D07E0E7C0C0
:104FD000E6FF0A0EE66EEFDDE552E5520001DE91D6
:104FE00039D0DEA311D00B0EE66EBBDDE552000119
:104FF000E85D07E0E8C0E6FF0B0EE66EDCDDE5529B
:10500000E5520001DE9326D0DEA511D00C0EE66E2F
:10501000A8DDE5520001E95D07E0E9C0E6FF0C0EFE
:10502000E66EC9DDE552E5520001DE9513D0DEA73C
:1050300011D00D0EE66E95DDE5520001EA5D07E048
:10504000EAC0E6FF0D0EE66EB6DDE552E552000160
:10505000DE9700D01200210EE66EE66892DDE55282
:04506000E552120003
:0C506400300EB16EA192A0820101016B20
:105070008C0E026FBF0E036F010E046F050E056FDD
:10508000030E066F0F0E0001EB150101006FE4D84F
:1050900001010E6B0B6B0F6B106B1200B190A192A4
:1050A0000101070706E003C1B3FF02C1B2FFB180EF
:1050B00049D00151020A2AE0030A01E043D003C1AA
:1050C000B3FF02C1B2FFB18008510807000913E025
:1050D0000CA105D0091D00150A11006F04D0005164
:1050E00009110A19006FB4EC2EF001010C910C4368
:1050F000020E076F0AD0091D00150A11006FB4ECEB
:105100002EF00101020E016F076F1CD00BA117D00A
:1051100003C1B3FF02C1B2FFB180005109110A19E6
:10512000006FB4EC2EF00101020E076F05C108F10B
:10513000010E016F0DC10CF10B6B108102D0016BE0
:105140000F8100D01200D9CFE6FFE1CFD9FF0101D6
:105150000BA103D0020E0E6F21D0F29E015117E178
:1051600003C1B3FF02C1B2FFB180005109110A1996
:10517000006FB4EC2EF0FE0EDBCF0CF10101010E3E
:10518000016F020E076F05C108F1108104D0FE0EF9
:10519000DBCF0DF10B81F28E0E6B00D0E552E7CF25
:1051A000D9FF1200D9CFE6FFE1CFD9FFFE0EDBCF4A
:1051B000EBF00001DE89F29E0F0E0001EB150101FC
:1051C000006F0001EB51010109150A6FB4EC2EF0DC
:1051D000F28EE552E7CFD9FF1200D9CFE6FFE1CF3B
:1051E000D9FFE652FE0EDB50DF6ED9CFE9FFDACFF2
:1051F000EAFFEF500F0B0101046F0451F66EF76ADE
:10520000D890F636F7363E0EF626630EF7220900E2
:10521000F5CF02F10A00F5CF03F1D9CFE9FFDACFDC
:10522000EAFFEF50300BE842E842E842E842050F5F
:10523000056FD9CFE9FFDACFEAFFEF50C00BE842A4
:10524000E842E842E842E842E842020F066FE552CF
:10525000E552E7CFD9FF1200010101510DE00F0E19
:105260000001EB150101006FB4EC2EF0B190A1929A
:105270000101016B0F810B6B0001A151F76A520F05
:10528000F66E630EF7220800F5CF09F10001EB512D
:10529000010109150A6F12000001EB5100D0120044
:1052A000D9CFE6FFE1CFD9FFE652DF6A01010B510A
:1052B000010B02E0000E01D0010E026ED9CFE9FF12
:1052C000DACFEAFF0250010BF36EFE0EEF14F3107B
:1052D000EF6E015102E1010E01D0000E026ED9CF36
:1052E000E9FFDACFEAFF0250010BF36EF346FD0E41
:1052F000EF14F310EF6EDF5000D0E552E552E7CF28
:10530000D9FF1200D9CFE6FFE1CFD9FFE652010164
:105310000451026ED9CFE9FFDACFEAFF02500F0B3A
:10532000F36EF00EEF14F310EF6E050E055D026ED6
:10533000D9CFE9FFDACFEAFF0250030BF36EF34651
:10534000F346F346F346CF0EEF14F310EF6E020E62
:10535000065D026ED9CFE9FFDACFEAFF0250030BF8
:10536000F36EF346F346F346F346F346F3463F0E39
:10537000EF14F310EF6EDF5000D0E552E552E7CFA7
:10538000D9FF120001010E5100D01200010110A13D
:1053900003D0106B010E07D00FA103D00F6B010ECD
:0853A00002D0000E00D0120043
:0853A80004011051600BE84202
:1053B000E842E842E842E842000901E055D01151D4
:1053C000070A51E00B0A4FE0070A40E0010A2CE00F
:1053D0000B0A28E0020A26E0030A22E0080A12E08B
:1053E000010A0EE00F0A0AE0030A01E03CD00101C5
:1053F000010E1B6F0101040E226F36D036D834D057
:1054000090D832D00101010E1B6F0101240E1C6FD8
:10541000010E1D6F010123930101010E206F24D0A5
:10542000A8D822D0EDD820D00101010E1B6F0401B5
:10543000145101011C6F1D6B250E1C27010E1D232D
:10544000010123930101010E206F0ED00101010E15
:105450001B6F04011451EA6A250FE96E010EEA225E
:1054600012C4EFFF01D000D01200800E0401105DC5
:1054700057E11351030A34E0010A10E0030A01E086
:105480004DD00101010E1B6F0101820E1C6F610ED8
:105490001D6F120E0101206F216B40D00101010E22
:1054A0001B6F04011251F66EF76AD890F636F73684
:1054B0001F0EF626620EF7220900F5CF1CF10A0036
:1054C000F5CF1DF1020E0101F76A1C25F66E1D5184
:1054D000F7220900F5CF20F10A00F5CF21F11ED007
:1054E0000101010E1B6F04011251F66EF76AD8908C
:1054F000F636F736230EF626620EF7220900F5CFB0
:105500001CF10A00F5CF1DF11CC1F6FF1DC1F7FF0C
:105510000800F5500101206F216B00D001012383A9
:1055200012000101010E1B6F0F0EE66E710EE66E8A
:105530000F0EE66E7DEC2EF0E552E552E552010EBF
:10554000E66E250EE66E010EE66E7DEC2EF0E5525F
:10555000E552E55212C424F10401125104E10101A3
:10556000050E226F05D00101060E226F47EC2DF0CB
:1055700012000401186B196B040110511F0B020A71
:105580000DE0030A07E0010A01E02CD00101010E41
:105590001B6F28D00101010E1B6F24D00101010EE9
:1055A0001B6F040114510F0B080DF350036A000F19
:1055B000026E040E03221451800B01E0010E040D53
:1055C000F350010102241E6F000E03201F6F1EC145
:1055D000E9FF1FC1EAFFEF50040B03E00401010ED5
:1055E000186F00D001011B050AE10101180E1C6FA4
:1055F000040E1D6F010123930101020E206F1200A2
:105600000401120510E110511F0B00090CE101010A
:10561000010E1B6F030E0401115D03E101012381E3
:1056200002D001012391040112513AE110511F0BE4
:10563000020836E114510F0B000932E00101010E9E
:105640001B6F040114510F0B080DF350036A000F78
:10565000026E040E03221451800B01E0010E040DB2
:10566000F350010102241E6F000E03201F6F030E72
:105670000401115D07E1840E1EC1E9FF1FC1EAFFAD
:10568000EF6E0ED014AF06D01EC1E9FF1FC1EAFFB6
:10569000EF6A06D0880E1EC1E9FF1FC1EAFFEF6E58
:0256A0001200F6
:0E56A2006C500BE1040100513C0BE842E84261
:1056B0000D0802E108D801D03CD804D0040E6C5C7F
:1056C00001E147D81200D9CFE6FFE1CFD9FFE6527A
:1056D00001011A6B1B6B206B216BD4EC29F0DF6A84
:1056E000DF50026E036A010E025C000E03581BE2DB
:1056F00001011B5101E017D0F76ADF34FE0BF736CA
:10570000F66E2B0EF626620EF7220900F5CF02F098
:105710000800F5CF03F004D003C0FAFF0250F96E81
:10572000FBDFDF2ADDD7DDD8E552E552E7CFD9FF31
:105730001200020E01011A5D0AE196D8040100BDB3
:1057400003D0C80E006F02D0880E006F01D00FD9B1
:105750001200040E0101225D0AE112C46EFF6E50B8
:10576000000803E2050E226F02D0030E226F010132
:105770001A050AE10BD8040104BD03D0C80E046F5A
:1057800002D0880E046F01D0F2D81200D9CFE6FF04
:10579000E1CFD9FF020EE1260101080E205D000EC7
:1057A000215905E220C1DEFF21C1DDFF03D0080E33
:1057B000DE6EDD6A040104930491010EDB500413D4
:1057C000DFCF05F4000EDB500101205F010EDB503E
:1057D000215B180E1E6F040E1F6F010123A31ED044
:1057E000D9CFE9FFDACFEAFFEE50ED1016E01CC189
:1057F000F6FF1DC1F7FF0800F5501EC1E9FF1FC1EC
:10580000EAFFEF6E01011E2B000E1F231C2B1D2330
:10581000DF06010E01E2DB06E3D71CD0D9CFE9FF9A
:10582000DACFEAFFEE50ED1015E01CC1E9FF1DC113
:10583000EAFFEF501EC1E9FF1FC1EAFFEF6E010151
:105840001E2B000E1F231C2B1D23DF06010E01E261
:10585000DB06E4D7020EE15C02E2E16AE552E16EAA
:10586000E552E7CFD9FF1200D9CFE6FFE1CFD9FF4C
:10587000020EE126030E04010015E76E010EE7CFCC
:10588000DBFF01C4DFFFDE5001012027DD502123B3
:10589000180E1C6F040E1D6FD9CFE9FFDACFEAFF97
:1058A000EE50ED1014E01CC1E9FF1DC1EAFFEF50FE
:1058B0001EC1E9FF1FC1EAFFEF6E1E2B000E1F2362
:1058C0001C2B1D23DF06010E01E2DB06E5D7020ECD
:1058D000E15C02E2E16AE552E16EE552E7CFD9FF11
:1058E00012006D9801011B510CE10401080E016FBB
:1058F000100E026F040E036F840E006F0401046F1C
:1059000035D0040110AF22D0010120510401165DF1
:10591000010121510401175904E216C420F117C4F2
:1059200021F134DF0101010E1A6F0401080E016F2D
:10593000100E026F040E036F800E006F0401180E2C
:10594000066F040E076FC80E046F10D00101020E1F
:105950001A6F0401056BC80E046F0401080E016F75
:10596000180E026F040E036FC80E006F12000101C3
:105970001A6B0401080E016F100E026F040E036F04
:0A598000880E006F0401046B120092
:06598A00040110511F0B87
:10599000010801E079D0145101E076D0060E115DC6
:1059A0002EE11351230A28E0010A13E0030A01E063
:1059B00024D00101020E1B6F0101240505E1010144
:1059C000A60E1C6F610E1D6F090E0101206F216B69
:1059D00014D00101020E1B6F0101240505E1010134
:1059E000FD0E1C6F610E1D6F0101240504E1220EE6
:1059F0000101206F216B01D000D00101238304013C
:105A00001051600BE842E842E842E842E8420108EF
:105A100001E03AD011510B0A31E0080A21E0090AED
:105A200019E0080A09E00B0A05E0080A01E02CD099
:105A30002CD82AD02BD828D00101020E1B6F0101CF
:105A4000260E1C6F010E1D6F010123930101010E33
:105A5000206F1AD00101020E1B6F13C426F114D05F
:105A60000101020E1B6F0101270E1C6F010E1D6F3D
:105A7000010123930101010E206F06D00101020EE6
:105A80001B6F12C427F100D0120012001200010196
:105A9000286B1E0E716E0401080E096F200E0A6F2E
:105AA000040E0B6F880E086F0401280E0E6F040E93
:105AB0000F6F400E0C6F1200D9CFE6FFE1CFD9FF78
:105AC000E652FC0EDB50080805E2080EF36EFC0EF1
:105AD000F3CFDBFFDF6AFC0EDB50DF5C19E2DF5047
:105AE000E76EFD0EDBCFE9FFFE0EDBCFEAFFE750EE
:105AF000E926000EEA22EF50E66EDF50EA6A280F30
:105B0000E96E040EEA22E552E750EF6EDF2AE3D792
:105B1000FC0EDBCF0DF4400E04010C170C7D880E3B
:105B20000C13E552E552E7CFD9FF1200D9CFE6FFBB
:105B3000E1CFD9FF0101286B040108BF31D0FC0E71
:105B4000DBCF02F00951D880025403E2FC0E09C4F5
:105B5000DBFF0101286BFC0EDB50285D19E22851A8
:105B6000EA6A200FE96E040EEA22EF50E66E285131
:105B7000E76EFD0EDBCFE9FFFE0EDBCFEAFFE7505D
:105B8000E926000EEA22E552E750EF6E282BE3D714
:105B90000401080E096F400E0817087D880E0813CF
:0E5BA0000101285100D0E552E7CFD9FF1200D5
:025BAE006DA6E2
:105BB0000CD80101220508E16DBA06D0686A696A4D
:105BC00069806988020E226F12006D6A696A6D86AB
:105BD0000101010E226F12006D6A696A0101226BD8
:105BE0001200ECEF2DF00101225101E13AD0685092
:105BF000040B04E06950040B01E03CD86DB231D0D5
:105C00006850010B04E06950010B01E054D8685062
:105C1000100B04E06950100B01E024D86850400BD1
:105C200004E06950400B01E03BD86850200B04E0D1
:105C30006950200B01E036D86850020B04E069502F
:105C4000020B01E036D8030E0101225D01E209D00A
:105C50006850080B06E06950080B03E051EC2BF08C
:105C600068961200698468986D82A19AF290F2B0E9
:105C700005D812006D92699468941200010123A165
:105C80000ED0F8DF6D840101080E296F070E2A6F10
:105C90002907000E2A5B29512A11FAE16D9412009E
:105CA000689C120070A003D0B7EC2CF07090689A3A
:105CB0001200689212006A6A686A9F0E6B6E7B0E11
:105CC000696E6E6A0F0EE66E710EE66E0F0EE66E70
:105CD00014D8E552E552E552160E706E68A602D051
:105CE0006896FCD76D98B7EC2CF001012391010167
:105CF000246B0101030E226F1200D9CFE6FFE1CF22
:105D0000D9FFFD0EDBCFE9FFFE0EDBCFEAFFFC0E75
:105D1000DB5004E0EE6AFC0EDB06F9D7E552E7CF74
:045D2000D9FF120095
:0C5D2400D9CFE6FFE1CFD9FF0101040E4A
:105D3000196FFE0EDBA602D08D8201D08D9200007D
:105D40000000010119078D80FE0EDBCFE7FFE79E03
:105D5000E746FE0EE7CFDBFF8D9001011951E9E127
:105D6000E552E7CFD9FF12000001EBA905D000C131
:105D7000E6FFD8DFE55204D018C1E6FFD3DFE552D5
:105D80000001DFAB05D0BAC0E6FFCCDFE55204D09E
:105D900017C1E6FFC7DFE55216C1E6FFC3DFE552D4
:105DA00015C1E6FFBFDFE5528D8400000000000052
:105DB0008D94120011C115F112C116F113C117F122
:105DC00014C118F1F29ED0DFF28E12000101116BA6
:105DD000126B136B146B156B166B176B186BB4EFA0
:105DE0002EF0D9CFE6FFE1CFD9FFFE0EDB500F0B2F
:105DF0000101116FFE0EDBB8DDDFE552E7CFD9FF01
:105E00001200D9CFE6FFE1CFD9FFFE0EDB500F0B1A
:105E10000101126FFE0EDBB8CDDFE552E7CFD9FFEF
:105E20001200D9CFE6FFE1CFD9FFFE0EDB500F0BFA
:105E30000101136FFE0EDBB8BDDFE552E7CFD9FFDE
:105E40001200D9CFE6FFE1CFD9FFFE0EDB500F0BDA
:105E50000101146FFE0EDBB8ADDFE552E7CFD9FFCD
:105E600012000101115100D012000101125100D0A5
:105E700012000101135100D012000101145100D091
:025E800012000E
:0E5E8200F02C52F2C8F61C5E2D6D1A2A7361C8
:105E90006A293F3E3C3830202123272F4755363191
:105EA0003B4C560611150902140B10041E0D120767
:105EB000050F161B0A08030C180E191D136824225F
:105EC000656C17FFFFFFFFBADB7C92DD6DE4573E88
:105ED00049C73EEE36D430F22BF3279F24CE2164FF
:105EE0001F4C1D771BDA196A182117F915ED14FAE2
:105EF000131B134F129411E7104710B20F270FA670
:105F00000E2D0EBC0D510DED0C8E0C350CE10B91D0
:105F10000B450BFC0AB80A770A380AFD09C4098E3A
:105F2000095A092809F808CA089E0873084B08236B
:105F300008FD07D907B607940773075307340717F7
:105F400007FA06DE06C306A9068F0676065E064732
:105F50000631061A060506F005DC05C805B505A2DA
:105F60000590057E056D055C054B053B052C051C64
:105F7000050D05FE04F004E204D404C704BA04AD20
:105F800004A004940488047C0470040000041080BD
:0B5F9000100000000008204008000086
:045F9C00D9CFE6FF74
:105FA000E1CFD9FFE652ECC0FAF0EDC0FBF0C26AD7
:105FB0003C0EC06EC280C282C2B2FED7C4CFFCF01B
:105FC0000001FB51C402F450DF6EFA51DF26DFCF2F
:105FD000E6FFB6EC10F0E5520001FE6B050EFD6F1A
:105FE000CD6A9E909D80D10ECF6E200ECE6ECD805C
:105FF000E552E552E7CFD9FF1200D9CFE6FFE1CF56
:10600000D9FFE652CD909E90D10ECF6E200ECE6E6F
:10601000CD80C2B23DD00001FC51C45C04E1FE6BF6
:10602000050EFD6F21D0FC51C45C10E2020EFE5D36
:1060300008E1C450FC5D026E040E025C02E3FD0741
:1060400004D0020EFE6F050EFD6F0ED0FE0508E1B6
:10605000FC51C45C026E040E025C02E3FD0704D036
:10606000010EFE6F050EFD6FFD5111E1FB51C402E3
:10607000F450DF6EFA51DF26DFCFE6FFC2EC10F0FE
:10608000E552C4CFFCF00001FE6B050EFD6FC2822D
:10609000E6EC15F034EC24F0E552E552E7CFD9FFF9
:0260A0001200EC
:0E60A200DACFE4FFE2CFDAFFE9CFE4FFEACF86
:1060B000E4FFF6CFE4FFF7CFE4FFF5CFE4FFF3CF43
:1060C000E4FFF4CFE4FFFACFE4FF00EE00F0020EAD
:1060D000E80403E3EECFE4FFFBD700EE02F0020E8C
:1060E000E80403E3EECFE4FFFBD7E6529EA002D024
:1060F000FDEC2FF0F050010B03E1F050020B02E039
:1061000064EC11F0F2A402D03EEC13F0A1A202D094
:106110004EEC28F0E55200EE03F0020EE80403E333
:10612000E5CFEDFFFBD700EE01F0020EE80403E33C
:10613000E5CFEDFFFBD7E5CFFAFFE5CFF4FFE5CFE5
:10614000F3FFE5CFF5FFE5CFF7FFE5CFF6FFE5CFAE
:10615000EAFFE5CFE9FFE5CFDAFF1100D8CFE4FF92
:10616000E0CFE4FFE46EDACFE4FFE2CFDAFFE652FD
:10617000E552E5CFDAFFE550E5CFE0FFE5CFD8FF08
:0261800010000D
:0E6182001201000200000008C0165E060100B7
:106190000102000109022900010100A032090400E6
:1061A000000203000003092101010001222200076F
:1061B0000581030800010705010308000104030924
:1061C000040A034B00310058004D00120353004FE6
:1061D0000032005200200042006F0078001203538A
:1061E000004F0032005200200043006F006E007428
:1061F0000072006F006C006C006500720006A0FF6A
:106200000901A1010903150026FF00750895028107
:10621000020904150026FF00750895029102C0943A
:0D622000619461BD61C161CB61DD618A598E
:02622E002A0E36
:10623000F66E200EF76E000EF86E00010900F550A4
:10624000F56F0900F550F66F03E1F56701D03DD019
:106250000900F550F06F0900F550F16F0900F55095
:10626000F26F09000900F550E96E0900F550EA6E79
:10627000090009000900F550F36F0900F550F46FAB
:1062800009000900F6CFF7F0F7CFF8F0F8CFF9F0F2
:10629000F0C0F6FFF1C0F7FFF2C0F8FF0001F353C2
:1062A00002E1F45307E00900F550EE6EF307F8E25F
:1062B000F407F9D7F7C0F6FFF8C0F7FFF9C0F8FF09
:0C62C0000001F507000EF65BBFD71200CE
:0462CC0007D8F28C71
:1062D000F28E10D83AEC1CF0FCD712000F0EC1124F
:1062E000140E6F6E0101226B0101236B0101246BFF
:1062F0000BEF1CF0D7EC2DF06FBE02D0F3EC2DF0BD
:02630000120089
:0E6302000008000400020001800020000400DA
:106310000100400010000800020000020103010219
:0263200004086F
:0E63220013EE00F023EE00F0F86A019C17EC79
:0E63300031F0B2EC31F066EC31F0FBD7120028
:02633E00D57A0E
:106340008CBF68C5AFCBF0D8B4E25EE578EC5AF10B
:066350003CF60102040806
:0A63560000EE00F00F0EEE6AEA629E
:04636000FDD7120053
:02636400120025
:00000001FF
